:10000000080C2500D00C02006607040A6606060AE2
:1000100061006607090A01022E00220C8E00030609
:10002000040A1B0C8E000306180A200CE501040AC2
:10003000D70C0200580289019C014306860A7C0005
:10004000690068007E007F007A00BA023F0C06005B
:10005000300C24006A00A3050509A30443062B0AFB
:100060000F0220003F0C84013F0E43063A0AA4020F
:10007000AA022B0A12024306010DFF0FA40432004C
:10008000A40513024306010DFF0F7500A4043300FD
:10009000A4051F02A4043600090C2400860A0802E5
:1000A000E20100080008000800080208030805082B
:1000B00007080A080D08120816081C082208290853
:1000C0003008380841084A0854085F086A0876086A
:1000D000830890089E08AD08BC08CC08DC08ED0831
:1000E000FF08090C2E00400003042F000F032D030E
:1000F0000306CC01EE02750A2C002C032D032C0301
:100100002D032C032D032C032D0300080400FF0CEA
:100110002D002E002F00090C24000B0C3D007F0049
:1001200047040000B50947069C0AD6096606C705BC
:1001300067066B069C0A4605FC0C3F024306AC0AA8
:10014000DF01FD02A80A0306200BBD0200008F0A92
:10015000DF020306F90B8F0A000000000000C7064B
:10016000BF02C704FE03900A260A66070008BF0202
:100170007E004705D60966070008BF0200001C0282
:10018000890138007802A706CE0A4F092900030426
:10019000E70629034704DF03B50A260A000000002A
:1001A00000000000000000000000CA0AC103E80AC5
:1001B00009029C004306040B0306E10ABC0212027A
:1001C000E40AFC001302870521000000000000087B
:1001D000FA02F50A060526051C02000000000000D0
:1001E000000000000000000000081A029C00070642
:1001F000FF0A0000030606040307060500080306BD
:100200002604030726050008870409026706F5028D
:100210000E0B3500D6066704460400086707F50391
:1002200000080B02670E100D3500D60667050008A2
:10023000100C8400070E4306F80BC706BF02240B00
:10024000090C3D00A4027F004704C704B509470616
:10025000300BD6096606C70567066106300B4604F3
:10026000FC0C3F024306180BDF01FD027A0B03066C
:10027000200B0A028B018C018D018E018F01430737
:10028000E20B6A026B026C026D026E02D609E40098
:10029000080C0600A4050A02EA07680B9801430748
:1002A000610B0B0299014307610B2C0C2400B4076E
:1002B000610B2706610BA3054F0A600B2706860A10
:1002C000740B0A02F00E700F4307860AA305E20AB8
:1002D00043065D0BB407900143065E0B1A027F0EC6
:1002E0002704430727058A014307610B2B0C2400D1
:1002F000A3054F0A00006003DF02230BFB0B8806F7
:100300001602A20B3E0243068E0B9E008F0B1102BB
:100310003D023F0743060706E706820B96002C00C6
:1003200003042C03180CEC01030C88002D00710948
:10033000090CAD00110203077F0B00000000CD0186
:100340000306160229006B0017024306D40B7F0E2A
:100350002A00F707AE0B040C8800B10B48021F0EF1
:1003600000002E008E076E06C30B2F004306BD0B48
:1003700003042A032B03EE02B90B17027F0E2F0092
:100380000A028F00D40B8A03070ECA012C00070C47
:100390008E002D0071090D022F002C032D032C035C
:1003A0002D03CD008F008A00F707DD0BC90103077D
:1003B00029000000A705A404860A89000306290075
:1003C000DA0B00000000000000000000D609000069
:1003D000000000000000000000000000000000001D
:1003E000860A00000000000000000000000000007D
:0C03F00000000000000000000000E10B15
:10040000840C2700310A800C060A830C2700A00CFC
:10041000C6042900080C2800E6046903C604030684
:10042000C6050000E605E8020C0A0000E60400002C
:10043000C60500000000E605C606E704E604E70777
:10044000470A07020F0EE2012B0A2E0A470A2B0A5F
:10045000310A360A470AA7020A02090AA7020F024E
:10046000090AE605C605A702A10C080AC605000090
:10047000E605080C2800E6050305C60703046F031C
:10048000E604C605E8023B0AE6050000E604C604E9
:10049000E6054A0A4B0AC605E7070008010880037B
:1004A0002F000F03070EE2017B0AD60B850B8D0B85
:1004B000510B490BFA0B2C0B2400070C4C01720951
:1004C0008C07690A6C062001FF0F6C0760010402AB
:1004D000F40A400143066F0A6C06170BFA0B6C070F
:1004E000170BFA0BE20101080208040808081008BB
:1004F000200840088008A006C90B0003070EE2018F
:10050000A90BFA0BFA0BB40BFA0BBB0BFA0BC20BD1
:100510005F078D0AFF06940AA40A7F07920A8706DE
:10052000940AA40A8007A40A07069D0A54069F0A93
:100530001F0786053F07A60400085406980A1F07F0
:1005400086043F07A60500081F0786043F07A60488
:10055000000847046704000F43063008010F4306F4
:100560003108030F43063208010F43063308070F13
:1005700043063608010F43063708150F43063808AF
:10058000010F43063908030F43063A080E0F4306CE
:1005900034082C0F43063B08010F43063C08030FA9
:1005A00043063D08040F43063E08090F43063F0873
:1005B0006705390F43060408010F43060D08670459
:1005C0004705FF0804020F0E0C0F43072C0B0B020C
:1005D000A9094706FA0B67066A07F00A3500350CC9
:1005E0004A075C0A6A070C0B0F0E2A000509000275
:1005F0008F014306A3044306280A00022F00D406F5
:10060000030BD405FC0B03094306030BA304280AC0
:100610000A02200040000F0B67062A0B0F0E2A006B
:10062000050900028F014307A3044307860AC30696
:100630001B0BC305FC0B310C2600060C2E006F00B3
:100640000400EF03210BEE021F0B6600C304A40499
:10065000A304860A8001130B0B02F90F4306080B53
:100660000A027D0F4306430B010F4306400B0A02AB
:10067000070ED501A9094706FA0B6A070C0BF40A05
:100680000A02070E3D0BEB0003046B034B0335001E
:10069000FA0B8007FA0B8003F00EA4043B010F0F46
:1006A000590B88098006340500020F0EA4043B0193
:1006B000F00F5B013B002F00A4055B014306640BB8
:1006C000BF0667054605690BDF06690BBF066704B1
:1006D00046040F025C014306750BFF055F06780BAD
:1006E0001F06730BA6058605780B1F068604FF04FC
:1006F0000F025D014306810B3F06A6053F07E70594
:10070000FA0B3F06A604E704FA0B14068F0BFA0651
:10071000910B0707950B0704AC0B1406870BFA0621
:10072000890B0706950B0705AC0BA70440031E0EAB
:1007300028008006080534070804340788090802E1
:100740004306B20BFD0E4306AC0B9406FA0BA30452
:10075000870B080C0600660006042604A4047A0031
:10076000BA027C006900FA0B740403077405340CA8
:1007700020001402F40AB4040307B405340C20006A
:100780001402F40A540403075405340C2000140224
:10079000F40A0C023A000002120F4306FA04010F99
:1007A0004306FA053A0C24001A02F40A00023F0F2D
:1007B0004307FA0BA402E006E50B1406E70BFA0662
:1007C000E90B0707ED0B0704AC0B1406DF0BFA0669
:1007D000E10B0706ED0B0705AC0B00032F000F0321
:1007E0001F0E280040039F07290034059F069F0B1A
:1007F000A705FA0BD404C304A304A404860A700C4E
:021FFE00E60FEC
:00000001FF
